:020000042000DA
:10000000084880F3088800F06FF900BF00BE0000C8
:1000100000BE00BE00BE00BF00BFFCE700BF00BFC7
:10002000FCE7000058280020D2B201E000F8012BC4
:10003000491EFBD270470022F6E710B513460A4668
:1000400004461946FFF7F0FF204610BD10B50246E2
:10005000002306E01468121D601C08B1002010BDCA
:100060001B1D8B42F6D30120F9E7000010B50020DC
:100070000F4908600EE00E4909684FF0006202EB7C
:10008000812000F075F80B49087009480068401C91
:10009000074908600648006807490968884203D292
:1000A000044800780428E6D001200449486010BDC7
:1000B0001006002018060020140600201C06002050
:1000C00038B5002024494860009002E00098401CA8
:1000D000009022480068401E0099884209D9009883
:1000E000401C4FF0006101EB80201B49C969884228
:1000F000ECD90EE04FF00062009902EB812000F095
:1001000037F804461648047004B938BD0098401CFE
:10011000009012480068401E009988420FD910488C
:10012000007804280BD10C48C0690B49096A0844BF
:100130004FF00062009902EB81218842DAD8012059
:10014000054948600A46116AD069FFF77FFF0249F6
:10015000486000BFD9E700001C06002014060020FC
:10016000180600200149C8607047000000200240C6
:1001700070B50546042440F6FF7000F085F804468B
:10018000042C19D10D48006940F002000B490861A8
:1001900008464561006940F04000086140F6FF7084
:1001A00000F072F80446012C06D00448006941F6BC
:1001B000FD71084001490861204670BD00200240E1
:1001C00004200B49C96801F0010109B101200EE0CA
:1001D0000749C96801F0040109B1022007E0044998
:1001E000C96801F0100109B1032000E00420704744
:1001F000002002400549096821F01001034A1160FE
:100200001146096801431160704700000020024058
:1002100070B505460E4604240F2000F035F804465C
:10022000042C13D10A48006940F001000849086114
:100230002E800F2000F028F80446012C06D0044838
:10024000006941F6FE71084001490861204670BD11
:10025000002002400549096801F03801034A116095
:1002600011460968014311607047000000200240F8
:1002700002480349486003484860704723016745C6
:1002800000200240AB89EFCD70B504460425FFF78E
:1002900097FF054605E000F0ACF9FFF791FF054632
:1002A000641E012D01D1002CF5D104B90525284685
:1002B00070BD000010B504200849087001200849ED
:1002C000087000F071F800F039F8FFF7D1FF8020D6
:1002D000044908603520FFF745FF10BD18060020CF
:1002E000190600201406002010B5FFF7E3FF12489E
:1002F000006830B1012807D0022808D003280CD1AB
:1003000008E000F02DF811E0FFF7B0FE0EE0FFF777
:10031000D7FE0BE000F056F908E042F23C01064837
:10032000FFF789FE00200449486000BF00BF00F0CD
:100330006DF900BF00BF10BD1C06002010B50021E4
:100340004FF0006000F002F810BD0000024A0A40C1
:100350000243024B1A60704780FFFF1F08ED00E068
:1003600070B50F48C46900F13C05002608E02988F3
:100370002046FFF74DFF0B490870A41CAD1CB61CAE
:100380000748006AB042F2D80120054948600A4691
:10039000116AD0693C3200F01BF90149486070BD18
:1003A0001C0600201806002010B5002400F038F8C4
:1003B0004FF4803000F08CF800F0E8F8174908702E
:1003C00008460078012827D1002000F075F80020A9
:1003D00000F0B0F84FF4806000F0A0F80220FFF7C2
:1003E00039FF1020FFF706FF4FF4E0114FF4803083
:1003F00000F0B2F8012000F0A9F800BF392000F0A9
:1004000035F80446002CF9D0022000F0B3F800BF04
:1004100000F04AF80828FBD110BD00001A060020A1
:100420000F48006840F001000D4908600846406828
:100430000C4908400A494860084600680A490840D3
:10044000074908600846006820F4802008600846D4
:10045000406820F4FE00486000208860704700007B
:10046000001002400000FFF8FFFFF6FE10B5014645
:100470000022002300204A11012A02D1094C2368DE
:1004800006E0022A02D1074C236A01E0054C636AA8
:1004900001F01F02012494401C400CB1012000E037
:1004A000002010BD001002400248406800F00C001F
:1004B000704700000010024001460020034A5068C7
:1004C00020F0F00008435060704700000010024028
:1004D0001149096821F480310F4A116011460968F9
:1004E00021F480211160B0F5803F03D0B0F5802F5A
:1004F0000ED106E00849096841F48031064A1160CE
:1005000007E00549096841F4A021034A116000E0B1
:1005100000BF00BF704700000010024001460020ED
:10052000034A506820F4E0600843506070470000C0
:100530000010024001460020034A506820F4605039
:1005400040EAC1005060704700100240014908664F
:10055000704700000000424202460020044B5868E9
:1005600020F47C1042EA01031843014B58607047A5
:100570000010024001460020034A506820F00300AA
:1005800008435060704700000010024038B500205A
:1005900000900024002500BF3120FFF767FF0546CB
:1005A0000098401C00901DB90098B0F5A06FF3D1E1
:1005B0003120FFF75BFF08B1012400E00024204652
:1005C00038BD000001200149486070471C0600202A
:1005D00070B50346002408E01D681B1D1668121D37
:1005E000B54201D0002070BD241D8C42F4D30120FF
:1005F000F9E708B500200090FF20009002E0009885
:10060000401E009000980028F9D108BD70470000F6
:0C061000FFFFFFFF80000000040101005C
:0400000520000001D6
:00000001FF
